:020000040800F2
:1000000000060020E1020008E3020008E302000805
:10001000E3020008E3020008E3020008E30200082C
:10002000E3020008E3020008E3020008C52200081A
:10003000E3020008E3020008E3020008E30200080C
:10004000E3020008E3020008E3020008E3020008FC
:10005000E3020008E3020008F12900081D2A000855
:10006000492A0008752A0008A12A0008DD0F0008A7
:1000700005100008311000085D1000088910000804
:10008000B1100008DD100008E3020008E3020008D8
:10009000E3020008E3020008E3020008CD2A00089A
:1000A000E3020008E3020008E3020008E30200089C
:1000B000E3020008E3020008E3020008E30200088C
:1000C000E3020008E3020008E3020008E30200087C
:1000D000E3020008E3020008E3020008E30200086C
:1000E000312B0008E3020008E3020008E3020008E5
:1000F000E3020008E3020008E30200080911000817
:10010000E3020008E3020008CD2B0008E302000828
:10011000E3020008E3020008E3020008E30200082B
:10012000351100085D11000889110008B51100089B
:10013000E1110008E3020008E3020008E3020008FE
:10014000E3020008E3020008E3020008E3020008FB
:10015000091200083512000861120008E3020008C5
:10016000E3020008E3020008E3020008E3020008DB
:10017000E3020008E3020008E3020008E3020008CB
:10018000E3020008E3020008A52B0008B92B0008D1
:10019000E3020008E3020008E3020008E3020008AB
:1001A000E3020008E3020008E3020008E30200089B
:1001B000E3020008E3020008E3020008E30200088B
:1001C000E3020008E3020008E3020008E30200087B
:1001D000E3020008E3020008E3020008E30200086B
:1001E000E3020008E3020008E3020008E30200085B
:1001F000E3020008E3020008E3020008E30200084B
:10020000E3020008E3020008E3020008E30200083A
:10021000E3020008E3020008E3020008E30200082A
:10022000E3020008E3020008E3020008E30200081A
:10023000E3020008E3020008E3020008E30200080A
:10024000E3020008E3020008E3020008E3020008FA
:10025000E3020008E3020008E3020008E3020008EA
:10026000E3020008E3020008E3020008E3020008DA
:10027000E3020008E3020008E3020008E3020008CA
:10028000E3020008E3020008E3020008E3020008BA
:10029000E3020008E3020008E3020008E3020008AA
:1002A000E3020008E3020008E3020008E30200089A
:1002B000E3020008E3020008E3020008E30200088A
:1002C000E3020008E3020008E3020008E30200087A
:1002D000E3020008E3020008E3020008E30200086A
:1002E00002E000F000F8FEE772B6374880F30888B5
:1002F000364880F3098836483649086040F20000E5
:10030000CCF200004EF63471CEF200010860BFF36B
:100310004F8FBFF36F8F40F20000C0F2F0004EF637
:100320008851CEF200010860BFF34F8FBFF36F8F8B
:100330004FF00000E1EE100A4EF63C71CEF20001E3
:100340000860062080F31488BFF36F8F02F01CF85A
:1003500002F01EF94FF055301F491B4A91423CBF35
:1003600041F8040BFAE71D49184A91423CBF41F895
:10037000040BFAE71A491B4A1B4B9A423EBF51F83D
:10038000040B42F8040BF8E700201849184A914280
:100390003CBF41F8040BFAE702F034F802F07EF9B2
:1003A000144C154DAC4203DA54F8041B8847F9E7A6
:1003B00000F042F8114C124DAC4203DA54F8041B21
:1003C0008847F9E702F01CB8000600200022002050
:1003D0000000000808ED00E00000002000060020FA
:1003E000602F000800220020302200203022002050
:1003F000F82F0020E0020008E0020008E0020008F8
:10040000E00200082DE9F04F2DED108AC1F80CD064
:10041000D0F80CD0BDEC108ABDE8F08F002383F338
:1004200011882846A047002001F006FCFEE701F0F5
:100430009FFB00DFFEE7000038B500F009FC00F08C
:1004400061FD01F0D7FE054601F032FF0446C0B958
:100450000E4B9D4217D001339D4242F2107512BFE0
:10046000044600250124002001F0CEFE0CB100F06E
:1004700075F800F01FFD284600F0F0F800F06EF867
:10048000F9E70025EFE70546EDE700BF010007B0FB
:1004900008B500F0A9FBA0F120035842584108BD5F
:1004A00007B541F21203022101A8ADF8043000F0B3
:1004B000B9FB03B05DF804FB38B5302383F3118832
:1004C000174803680BB101F075FC0023154A4FF47F
:1004D0007A71134801F064FC002383F31188124CF5
:1004E000236813B12368013B2360636813B1636819
:1004F000013B63600D4D2B7833B963687BB90220F3
:1005000000F06EFC322363602B78032B07D1636805
:100510002BB9022000F064FC4FF47A73636038BD9D
:1005200030220020B9040008502300204822002077
:10053000084B187003280CD8DFE800F00805020803
:10054000022000F043BC022000F036BC024B002227
:100550005A6070474822002050230020F8B5394BDC
:10056000394A1C46196801316BD004339342F9D1E2
:100570006268364B9A4264D9354B9B6803F100633D
:1005800003F500339A425CD2002000F087FB022082
:10059000FFF7CEFF2F4B00219A6C99641A6F1967F1
:1005A0001A6FDA6CD9645A6F59675A6F1A6D1965E8
:1005B0009A6F99679B6F72B64FF0E023C3F8084DAE
:1005C000D4E90004BFF34F8FBFF36F8F224AC2F804
:1005D0008410BFF34F8F536923F480335361BFF30B
:1005E0004F8FD2F8803043F6E076C3F3C905C3F3EA
:1005F0004E335B0103EA060C29464CEA8177013948
:10060000C2F87472F9D2203B13F1200FF2D1BFF37C
:100610004F8FBFF36F8FBFF34F8FBFF36F8F536950
:1006200023F4003353610023C2F85032BFF34F8FDD
:10063000BFF36F8F302383F31188854680F30888DA
:100640002047F8BD0000020820000208FFFF010853
:10065000002200200045025800ED00E02DE9F04F97
:1006600093B0B44B2022FF2100900AA89D6800F0AF
:10067000CBFBB14A1378A3B90121B04811700360D4
:10068000302383F3118803680BB101F093FB00233F
:10069000AB4A4FF47A71A94801F082FB002383F33F
:1006A0001188009B13B1A74B009A1A60A64A1378D1
:1006B000032B03D000231370A24A53604FF0000AAB
:1006C000009CD3465646D146012000F07FFB24B162
:1006D0009C4B1B68002B00F02682002000F084FA5F
:1006E0000390039B002BF2DB012000F065FB039BD2
:1006F000213B1F2BE8D801A252F823F07D07000808
:10070000A507000839080008C9060008C90600083E
:10071000C9060008CB0800089B0A0008B5090008B4
:10072000170A00083F0A0008650A0008C906000801
:10073000770A0008C9060008E90A00081D08000831
:10074000C90600082D0B0008890700081D080008CD
:10075000C9060008170A0008C9060008C9060008EB
:10076000C9060008C9060008C9060008C90600082D
:10077000C9060008C9060008390800080220FFF76A
:1007800087FE002840F0F981009B022105A8BAF1FC
:10079000000F08BF1C4641F21233ADF8143000F0D0
:1007A00041FA91E74FF47A7000F01EFA071EEBDB76
:1007B0000220FFF76DFE0028E6D0013F052F00F272
:1007C000DE81DFE807F0030A0D101336052304214C
:1007D00005A8059300F026FA17E004215548F9E72B
:1007E00004215A48F6E704215948F3E74FF01C0862
:1007F000404608F1040800F053FA0421059005A8CA
:1008000000F010FAB8F12C0FF2D101204FF00009DE
:1008100000FA07F747EA0B0B5FFA8BFB00F040FB8F
:1008200026B10BF00B030B2B08BF0024FFF738FE9B
:100830004AE704214748CDE7002EA5D00BF00B0373
:100840000B2BA1D10220FFF723FE074600289BD0E7
:100850000120002600F022FA0220FFF769FE1FFAAD
:1008600086F8404600F02AFA0446B0B103994046A3
:100870000136A1F140025142514100F02FFA002807
:10088000EDD1BA46044641F21213022105A83E46B4
:10089000ADF8143000F0C6F916E725460120FFF741
:1008A00047FE244B9B68AB4207D9284600F0F8F975
:1008B000013040F067810435F3E70025224BBA464A
:1008C0003E461D701F4B5D60A8E7002E3FF45CAFF5
:1008D0000BF00B030B2B7FF457AF0220FFF728FE22
:1008E000322000F081F9B0F10008FFF64DAF18F0AA
:1008F00003077FF449AF0F4A08EB05039268934260
:100900003FF642AFB8F5807F3FF73EAF124BB84598
:10091000019323DD4FF47A7000F066F90390039A97
:10092000002AFFF631AF039A0137019B03F8012B30
:10093000EDE700BF002200204C23002030220020E1
:10094000B90400085023002048220020042200207F
:10095000082200200C2200204C220020C820FFF793
:1009600097FD074600283FF40FAF1F2D11D8C5F1A2
:1009700020020AAB25F0030084494245184428BFF1
:100980004246019200F036FA019AFF217F4800F0BA
:100990003BFA4FEAA803C8F387027C492846019333
:1009A00000F03AFA064600283FF46DAF019B05EBD4
:1009B000830533E70220FFF76BFD00283FF4E4AE28
:1009C00000F0AAF900283FF4DFAE0027B846704BCC
:1009D0009B68BB4218D91F2F11D80A9B01330ED038
:1009E00027F0030312AA134453F8203C0593404612
:1009F000042205A9043700F0DBFA8046E7E7384611
:100A000000F04EF90590F2E7CDF81480042105A816
:100A100000F008F902E70023642104A8049300F021
:100A2000F7F800287FF4B0AE0220FFF731FD002870
:100A30003FF4AAAE049800F065F90590E6E70023BC
:100A4000642104A8049300F0E3F800287FF49CAE2E
:100A50000220FFF71DFD00283FF496AE049800F039
:100A600053F9EAE70220FFF713FD00283FF48CAEAC
:100A700000F062F9E1E70220FFF70AFD00283FF4E9
:100A800083AE05A9142000F05DF907460421049007
:100A900004A800F0C7F83946B9E7322000F0A4F8FE
:100AA000071EFFF671AEBB077FF46EAE384A07EB48
:100AB0000903926893423FF667AE0220FFF7E8FC15
:100AC00000283FF461AE27F003074F44B9453FF4D7
:100AD000A5AE484609F1040900F0E2F804210590AA
:100AE00005A800F09FF8F1E74FF47A70FFF7D0FC0B
:100AF00000283FF449AE00F00FF9002844D00A9BCB
:100B000001330BD008220AA9002000F085F9002843
:100B10003AD02022FF210AA800F076F9FFF7C0FCA6
:100B20001C4801F08FF813B0BDE8F08F002E3FF4A1
:100B30002BAE0BF00B030B2B7FF426AE00236421AE
:100B400005A8059300F064F8074600287FF41CAE62
:100B50000220FFF79DFC804600283FF415AEFFF70A
:100B60009FFC41F2883001F06DF8059800F0B0F973
:100B700046463C4600F094F9A6E506464EE64FF0A0
:100B8000000901E6BA467EE637467CE64C220020A4
:100B900000220020A0860100104B70B51B780C4687
:100BA0000133DBB2012B12D80D4B1D684FF47A7361
:100BB0002968A2FB033222460E6A01462846B04746
:100BC000844204D1074B002201201A7070BD4FF4FB
:100BD000FA7001F037F80020F8E700BF102200207B
:100BE000142200209C230020002307B50246012187
:100BF0000DF107008DF80730FFF7CEFF20B19DF80B
:100C0000070003B05DF804FB4FF0FF30F9E7000088
:100C10000A46042108B5FFF7BFFF80F00100C0B20B
:100C2000404208BD074B0A4630B41978064B53F8CA
:100C30002140014623682046DD69044BAC4630BCA8
:100C4000604700BF9C23002014220020A0860100E2
:100C500070B5104C0025104E01F0B4F920803068BA
:100C6000238883420CD800252088013801F0A6F99A
:100C700023880544013BB5F5802F2380F4D370BD54
:100C800001F09CF9336805440133B5F5003F33604A
:100C9000E5D3E8E79E2300205823002001F060BA46
:100CA00000F1006000F500300068704700F100605E
:100CB000920000F5003001F0E1B90000054B1A6820
:100CC000054B1B889B1A834202D9104401F076B968
:100CD00000207047582300209E23002038B504468A
:100CE000074D29B128682044BDE8384001F07EB99D
:100CF0002868204401F068F90028F3D038BD00BF0F
:100D0000582300200020704700F1FF5000F58F109D
:100D1000D0F8000870470000064991F8243033B13C
:100D200000230822086A81F82430FFF7BFBF0120A2
:100D3000704700BF5C230020014B1868704700BF5C
:100D40000010005C194B01380322084470B51D687F
:100D5000174BC5F30B042D0C1E88A6420BD15C6803
:100D60000A46013C824213460FD214F9016F4EB17C
:100D700002F8016BF6E7013A03F10803ECD1814276
:100D80000B4602D22C2203F8012B0424094A1688B0
:100D9000AE4204D1984284BF967803F8016B013CBF
:100DA00002F10402F3D1581A70BD00BF0010005CBC
:100DB00018220020C02C0008022803D1024B4FF05B
:100DC00080629A61704700BF000C0258022803D16C
:100DD000024B4FF480629A61704700BF000C0258CA
:100DE000022804D1024A536983F480635361704737
:100DF000000C0258002310B5934203D0CC5CC454BD
:100E00000133F9E710BD000002440346934202D0CB
:100E100003F8011BFAE770472DE9F8431F4D14460C
:100E20000746884695F8242052BBDFF870909CB3A3
:100E300095F824302BB92022FF2148462F62FFF776
:100E4000E3FF95F824004146C0F1080205EB80005D
:100E5000A24228BF2246D6B29200FFF7CBFF95F8F8
:100E60002430A41B17441E449044E4B2F6B2082E6A
:100E700085F82460DBD1FFF74FFF0028D7D108E0C9
:100E80002B6A03EB82038342CFD0FFF745FF002894
:100E9000CBD10020BDE8F8830120FBE75C230020D4
:100EA000024B1A78024B1A70704700BF9C23002037
:100EB00010220020034B04490B60044B186800F01B
:100EC000BDBD00BF80841E008423002014220020AA
:100ED000094B1822002110B504461846FFF794FF6D
:100EE000064A074B01461278046053F82200BDE819
:100EF000104000F0A3BD00BF842300209C230020ED
:100F000014220020F0B5A1B071B600230120002406
:100F100080261A46194600F041FA4FF4D067214A5C
:100F20003D25136923BBD2F810310BBB036804F1D4
:100F3000006199600368C3F80CD003685E600368C1
:100F40001F6001680B6843F001030B6001680B68C8
:100F500023F01E030B6001680B68DB07FCD4037BE6
:100F60008034416805FA03F3B4F5001F0B60D8D153
:100F700000F04AFAB4F5001F11D000240A4E0B4DC0
:100F8000012001F0EDF83388A34205D928682044F8
:100F9000013401F02BF8F6E7002001F0E1F861B62A
:100FA00021B0F0BD002000529E23002058230020D5
:100FB00030B50A44084D91420DD011F8013B58401C
:100FC000082340F30004013B2C4013F0FF0384EAA4
:100FD0005000F6D1EFE730BD2083B8ED08B5074BE0
:100FE000074A196801F03D01996053680BB1906898
:100FF0009847BDE8084001F09DB900BF00000240DD
:10100000A023002008B5084B1968890901F03D01AB
:101010008A019A60054AD3680BB110699847BDE808
:10102000084001F087B900BF00000240A023002063
:1010300008B5084B1968090C01F03D010A049A60D3
:10104000054A53690BB190699847BDE8084001F023
:1010500071B900BF00000240A023002008B5084B72
:101060001968890D01F03D018A059A60054AD36926
:101070000BB1106A9847BDE8084001F05BB900BFAA
:1010800000000240A023002008B5074B074A59681A
:1010900001F03D01D960536A0BB1906A9847BDE8F1
:1010A000084001F047B900BF00000240A023002023
:1010B00008B5084B5968890901F03D018A01DA60D9
:1010C000054AD36A0BB1106B9847BDE8084001F0A0
:1010D00031B900BF00000240A023002008B5084B32
:1010E0005968090C01F03D010A04DA60054A536BA6
:1010F0000BB1906B9847BDE8084001F01BB900BFE9
:1011000000000240A023002008B5084B5968890D53
:1011100001F03D018A05DA60054AD36B0BB1106C12
:101120009847BDE8084001F005B900BF0000024043
:10113000A023002008B5074B074A196801F03D01BC
:101140009960536C0BB1906C9847BDE8084001F072
:10115000F1B800BF00040240A023002008B5084BEE
:101160001968890901F03D018A019A60054AD36C2A
:101170000BB1106D9847BDE8084001F0DBB800BF27
:1011800000040240A023002008B5084B1968090C90
:1011900001F03D010A049A60054A536D0BB1906D50
:1011A0009847BDE8084001F0C5B800BF0004024000
:1011B000A023002008B5084B1968890D01F03D01F6
:1011C0008A059A60054AD36D0BB1106E9847BDE849
:1011D000084001F0AFB800BF00040240A023002087
:1011E00008B5074B074A596801F03D01D960536EB5
:1011F0000BB1906E9847BDE8084001F09BB800BF66
:1012000000040240A023002008B5084B5968890952
:1012100001F03D018A01DA60054AD36E0BB1106F0F
:101220009847BDE8084001F085B800BF00040240BF
:10123000A023002008B5084B5968090C01F03D01B6
:101240000A04DA60054A536F0BB1906F9847BDE806
:10125000084001F06FB800BF00040240A023002046
:1012600008B5084B5968890D01F03D018A05DA601F
:10127000054AD36F13B1D2F880009847BDE8084003
:1012800001F058B800040240A023002000230C49BC
:1012900010B51A460B4C0B6054F82300026001EBAA
:1012A000430004334260402BF6D1074A4FF0FF332E
:1012B0009360D360C2F80834C2F80C3410BD00BF8C
:1012C000A0230020D02C0008000002400F28F8B511
:1012D00010D9102810D0112811D0122808D10F24AD
:1012E0000720DFF8B4E00126DEF80050A04208D95C
:1012F000002649E00446F4E70F240020F1E7072424
:10130000FBE706FA00F73D4240D1214C4FEA001CB2
:101310003D4304EB00160EEBC000CEF80050C0E9D0
:101320000123FBB24BB11B48836B43F00103836382
:10133000036E43F001030366036E17F47F4F09D079
:101340001448836B43F002038363036E43F002038C
:101350000366036E54F80C00036823F01F03036058
:10136000056815F00105FBD104EB0C033D2493F84F
:101370000CC05F6804FA0CF43C60212405604461F1
:1013800012B1987B00F08EF93046F8BD0130ADE720
:10139000D02C000800450258A023002010B53024AE
:1013A00084F31188FFF792FF002383F3118810BDA7
:1013B00010B50446807B00F08BF901231049627B55
:1013C00003FA02F20B6823EA0203DAB20B604AB9AD
:1013D0000C4A916B21F001019163116E21F0010122
:1013E0001166126E13F47F4F09D1064B9A6B22F0EF
:1013F00002029A631A6E22F002021A661B6E10BD78
:10140000A02300200045025808B5302383F311883B
:10141000FFF7CEFF002383F3118808BD02684368FD
:101420001143016003B1184770470000024A136876
:1014300043F0C0031360704700780040024A13680D
:1014400043F0C00313607047007C004037B51A4C6E
:101450001A4D204600F0E6FA04F11400009400232F
:101460004FF40072164900F0A3F94FF400721549C9
:1014700004F138000094144B00F01CFA134BC4E93B
:101480001735134C204600F0CDFA04F11400002368
:101490004FF400720F49009400F08AF90E4B4FF49C
:1014A00000720E4904F13800009400F003FA0C4B6E
:1014B000C4E9173503B030BD2424002000E1F50550
:1014C000FC240020FC2800202D1400080078004097
:1014D00090240020FC2600203D140008FC2A002057
:1014E000007C0040037C30B5274C002918BF0C4617
:1014F000012B0CD1254B984236D1254B9A6C42F0EA
:1015000080429A641A6F42F080421A671B6F226809
:10151000036EC16D03EB52038466B3FBF2F36268A2
:10152000150442BF23F0070503F0070343EA450310
:10153000CB60A36843F040034B60E36843F00103D2
:101540008B6042F4967343F001030B604FF0FF335E
:101550000B62510505D512F0102211D0B2F1805F57
:1015600010D080F8643030BD0A4B9842CFD1084B80
:101570009A6C42F000429A641A6F42F00042C4E74B
:101580007F23EEE73F23ECE7D02D00082424002042
:1015900000450258902400202DE9F047C66D05460D
:1015A0003768F469210734621AD014F0080118BFB3
:1015B0004FF48071E20748BF41F02001A3074FF0CC
:1015C000300348BF41F04001600748BF41F080014F
:1015D00083F31188281DFFF721FF002383F311886F
:1015E000E2050AD5302383F311884FF48061281D6A
:1015F000FFF714FF002383F311884FF030094FF0F9
:10160000000A14F0200838D13B0616D54FF03009F7
:1016100005F1380A200610D589F31188504600F0EC
:101620007DF9002836DA0821281DFFF7F7FE27F09C
:1016300080033360002383F31188790614D5620692
:1016400012D5302383F31188D5E913239A4208D1A8
:101650002B6C33B127F040071021281DFFF7DEFE69
:101660003760002383F31188E30618D5AA6E136947
:10167000ABB15069BDE8F047184789F31188736A28
:10168000284695F86410194000F0E6F98AF31188AD
:10169000F469B6E7B06288F31188F469BAE7BDE887
:1016A000F0870000090100F16043012203F5614366
:1016B000C9B283F8001300F01F039A4043099B004E
:1016C00003F1604303F56143C3F880211A6070475A
:1016D00000F01F0301229A40430900F160409B0083
:1016E00000F5614003F1604303F56143C3F88020D6
:1016F000C3F88021002380F800337047F8B5154601
:10170000826804460B46AA4200D28568A169266910
:10171000761AB5420BD218462A46FFF76BFBA3692F
:101720002B44A3612846A3685B1BA360F8BD0CD9BA
:10173000AF1B18463246FFF75DFB3A46E16830447E
:10174000FFF758FBE3683B44EBE718462A46FFF7F0
:1017500051FBE368E5E7000083689342F7B5044670
:10176000154600D28568D4E90460361AB5420BD21A
:101770002A46FFF73FFB63692B4463612846A36851
:101780005B1BA36003B0F0BD0DD93246AF1B0191C6
:10179000FFF730FB01993A46E0683144FFF72AFB36
:1017A000E3683B44E9E72A46FFF724FBE368E4E704
:1017B00010B50A440024C361029B8460C1600261C9
:1017C0000362C0E90000C0E9051110BD08B5D0E909
:1017D0000532934201D1826882B982680132826007
:1017E0005A1C426119700021D0E904329A4224BF88
:1017F000C368436100F042FA002008BD4FF0FF309B
:10180000FBE7000070B5302304460E4683F31188D1
:10181000A568A5B1A368A269013BA360531CA3619D
:1018200015782269934224BFE368A361E3690BB191
:1018300020469847002383F31188284607E0314665
:10184000204600F00BFA0028E2DA85F3118870BD1B
:101850002DE9F74F04460E4617469846D0F81C90DF
:101860004FF0300A8AF311884FF0000B154665B12E
:101870002A4631462046FFF741FF034660B94146FC
:10188000204600F0EBF90028F1D0002383F3118803
:10189000781B03B0BDE8F08FB9F1000F03D00190C1
:1018A0002046C847019B8BF31188ED1A1E448AF32A
:1018B0001188DCE7C160C361009B82600362C0E9FC
:1018C00005111144C0E9000001617047F8B50446F4
:1018D0000D461646302383F31188A768A7B1A36885
:1018E000013BA36063695A1C62611D70D4E9043234
:1018F0009A4224BFE3686361E3690BB120469847CD
:10190000002080F3118807E03146204600F0A6F958
:101910000028E2DA87F31188F8BD0000D0E905233A
:1019200010B59A4201D182687AB9826800210132E9
:1019300082605A1C82611C7803699A4224BFC36882
:10194000836100F09BF9204610BD4FF0FF30FBE7AC
:101950002DE9F74F04460E4617469846D0F81C90DE
:101960004FF0300A8AF311884FF0000B154665B12D
:101970002A4631462046FFF7EFFE034660B941464E
:10198000204600F06BF90028F1D0002383F3118882
:10199000781B03B0BDE8F08FB9F1000F03D00190C0
:1019A0002046C847019B8BF31188ED1A1E448AF329
:1019B0001188DCE7026843681143016003B11847EE
:1019C000704700001430FFF743BF00004FF0FF33B3
:1019D0001430FFF73DBF00003830FFF7B9BF0000FB
:1019E0004FF0FF333830FFF7B3BF00001430FFF77C
:1019F00009BF00004FF0FF311430FFF703BF0000B4
:101A00003830FFF763BF00004FF0FF323830FFF788
:101A10005DBF0000012914BF6FF013000020704764
:101A2000FFF714BD044B036000234360C0E9023399
:101A300001230374704700BFE82D000810B5302360
:101A4000044683F31188FFF74DFD02230020237421
:101A500080F3118810BD000038B5C36904460D46F7
:101A60001BB904210844FFF7A5FF294604F114001F
:101A7000FFF7ACFE002806DA201D4FF40061BDE838
:101A80003840FFF797BF38BD0023826803750369AC
:101A90001B6899689142FBD25A68036042601060EB
:101AA0005860704700238268037503691B68996852
:101AB0009142FBD85A6803604260106058607047DA
:101AC00008B50846302383F311880B7D032B05D01E
:101AD000042B0DD02BB983F3118808BD8B6900222C
:101AE0001A604FF0FF338361FFF7CEFF0023F2E768
:101AF000D1E9003213605A60F3E70000FFF7C4BF7A
:101B0000054BD96808751868026853601A6001228D
:101B1000D8600275FEF776BC002D00200C4B30B566
:101B2000DD684B1C87B004460FD02B46094A684637
:101B300000F036F92046FFF7E3FF009B13B168463B
:101B400000F038F9A86907B030BDFFF7D9FFF9E711
:101B5000002D0020C11A0008044B1A68DB68906849
:101B60009B68984294BF002001207047002D002000
:101B7000084B10B51C68D868226853601A600122AF
:101B8000DC602275FFF78EFF01462046BDE810405D
:101B9000FEF738BC002D002038B5074C0123002586
:101BA000064907482370656000F09AFC0223237001
:101BB00085F3118838BD00BF682F0020142E00085F
:101BC000002D002000F02CB98B600223086108462C
:101BD0008B8270478368A3F1840243F8142C026956
:101BE00043F8442C426943F8402C094A43F8242C1A
:101BF000C268A3F1200043F8182C022203F80C2C31
:101C0000002203F80B2C034A43F8102C704700BF46
:101C10001D040008002D002008B5FFF7DBFFBDE81C
:101C20000840FFF76BBF0000024BDB6898610F2094
:101C3000FFF766BF002D0020302383F31188FFF7E4
:101C4000F3BF000008B50146302383F31188082054
:101C5000FFF764FF002383F3118808BD064BDB68A0
:101C600039B1426818605A60136043600420FFF77E
:101C700055BF4FF0FF307047002D00200368984299
:101C800006D01A680260506018469961FFF736BFA7
:101C900070470000036810B59C68A2420CD85C68CD
:101CA0008A600B604C602160596099688A1A9A605A
:101CB0004FF0FF33836010BD121B1B68ECE7000080
:101CC0000A2938BF0A2170B504460D460A26601954
:101CD00000F0FEFB00F0E6FB041BA54203D8751CD8
:101CE00004462E46F3E70A2E04D90120BDE87040D1
:101CF00000F036BC70BD0000F8B5144B0D460A2A42
:101D00004FF00A07D96103F11001826038BF0A223F
:101D1000416019691446016048601861A81800F014
:101D2000C7FB00F0BFFB431B0646A34206D37C1C47
:101D300028192746354600F0CBFBF2E70A2F04D9D5
:101D40000120BDE8F84000F00BBCF8BD002D0020DC
:101D5000F8B506460D4600F0A5FB0F4A134653F8AA
:101D6000107F9F4206D12A4601463046BDE8F84022
:101D7000FFF7C2BFD169BB68441A2C1928BF2C4693
:101D8000A34202D92946FFF79BFF2246314603486A
:101D9000BDE8F840FFF77EBF002D0020102D002089
:101DA000C0E90323002310B45DF8044B4361FFF73F
:101DB000CFBF000010B5194C236998420DD081683F
:101DC000D0E9003213605A609A680A449A6000238E
:101DD00003604FF0FF33A36110BD0268234643F850
:101DE000102F53600022026022699A4203D1BDE89D
:101DF000104000F067BB936881680B44936000F06B
:101E000051FB2269E1699268441AA242E4D9114463
:101E1000BDE81040091AFFF753BF00BF002D002096
:101E20002DE9F047DFF8BC8008F110072C4ED8F8F8
:101E3000105000F037FBD8F81C40AA68031B9A42E8
:101E40003ED814444FF00009D5E90032C8F81C40D0
:101E500013605A60C5F80090D8F81030B34201D131
:101E600000F030FB89F31188D5E903312846984703
:101E7000302383F311886B69002BD8D000F012FB5C
:101E80006A69A0EB040982464A450DD2022000F09F
:101E900067FB0022D8F81030B34208D151462846DB
:101EA000BDE8F047FFF728BF121A2244F2E712EB11
:101EB00009092946384638BF4A46FFF7EBFEB5E721
:101EC000D8F81030B34208D01444C8F81C00211AC6
:101ED000A960BDE8F047FFF7F3BEBDE8F08700BF9B
:101EE000102D0020002D002000207047FEE700008C
:101EF000704700004FF0FF3070470000BFF34F8F76
:101F0000044B1A695107FCD1D3F810215207F8D1BC
:101F1000704700BF0020005208B50D4B1B78ABB9CD
:101F2000FFF7ECFF0B4BDA68D10704D50A4A5A6079
:101F300002F188325A60D3F80C21D20706D5064A3E
:101F4000C3F8042102F18832C3F8042108BD00BFA0
:101F5000702F0020002000522301674508B5114B67
:101F60001B78F3B9104B1A69510703D5DA6842F0B0
:101F70004002DA60D3F81021520705D5D3F80C21BE
:101F800042F04002C3F80C21FFF7B8FF064BDA68B5
:101F900042F00102DA60D3F80C2142F00102C3F8EA
:101FA0000C2108BD702F0020002000520F289ABF7E
:101FB00000F5806040040020704700004FF40030BE
:101FC00070470000102070470F2808B50BD8FFF7A6
:101FD000EDFF00F500330268013204D10430834282
:101FE000F9D1012008BD0020FCE700000F2838B51A
:101FF00005463FD8FFF782FF1F4CFFF78DFF4FF0DC
:10200000FF3307286361C4F814311DD82361FFF73B
:1020100075FF030243F02403E360E36843F08003A9
:10202000E36023695A07FCD42846FFF767FFFFF7F0
:10203000BDFF4FF4003100F0F5F82846FFF78EFFA2
:10204000BDE83840FFF7C0BFC4F81031FFF756FFB6
:10205000A0F108031B0243F02403C4F80C31D4F8A8
:102060000C3143F08003C4F80C31D4F810315B0715
:10207000FBD4D9E7002038BD002000522DE9F84FED
:1020800005460C46104645EA0203DE0602D0002053
:10209000BDE8F88F20F01F00DFF8BCB0DFF8BCA06F
:1020A000FFF73AFF04EB0008444503D10120FFF796
:1020B00055FFEDE720222946204600F0DBFD10B950
:1020C00020352034F0E72B4605F120021F68791CEB
:1020D000DDD104339A42F9D105F178431B481C4EF7
:1020E000B3F5801F1B4B38BF184603F1F80332BF0E
:1020F000D946D1461E46FFF701FF0760A5EB040C49
:10210000336804F11C0143F002033360231FD9F844
:10211000007017F00507FAD153F8042F8B424CF8E2
:102120000320F4D1BFF34F8FFFF7E8FE4FF0FF33EA
:102130002022214603602846336823F002033360DF
:1021400000F098FD0028BBD03846B0E714210052BB
:102150000C20005214200052102000521021005276
:1021600010B5084C237828B11BB9FFF7D5FE012321
:10217000237010BD002BFCD02070BDE81040FFF78D
:10218000EDBE00BF702F00200244074BD2B210B545
:10219000904200D110BD441C00B253F8200041F819
:1021A000040BE0B2F4E700BF504000580E4B30B5CE
:1021B0001C6F240405D41C6F1C671C6F44F400447E
:1021C0001C670A4C02442368D2B243F48073236034
:1021D000074B904200D130BD441C51F8045B00B263
:1021E00043F82050E0B2F4E7004402580048025897
:1021F0005040005807B5012201A90020FFF7C4FF95
:10220000019803B05DF804FB13B50446FFF7F2FF35
:10221000A04205D0012201A900200194FFF7C6FFCA
:1022200002B010BD0144BFF34F8F064B884204D368
:10223000BFF34F8FBFF36F8F7047C3F85C0220303E
:10224000F4E700BF00ED00E0114BDA6952021ED541
:102250009A69D00704D50F4A9A6002F144329A6015
:102260000B4BDA69D107FCD41A6A22F480021A6295
:102270009A6942F002029A61DA69D207FCD49A693B
:1022800042F001029A61024AD369DB07FCD470472D
:10229000002000523B2A1908034B1A681AB9034A56
:1022A000D2F8D0241A607047742F002000400258E2
:1022B00008B5FFF7F1FF024B1868C0F3806008BD56
:1022C000742F0020EFF30983054968334A6B22F02D
:1022D00001024A6383F30988002383F3118870475E
:1022E00000EF00E0302080F3118862B60D4B0E4AFB
:1022F000D96821F4E0610904090C0A430B49DA604A
:10230000D3F8FC2042F08072C3F8FC20084AC2F8DF
:10231000B01F116841F0010111602022DA7783F8C3
:102320002200704700ED00E00003FA0555CEACC571
:10233000001000E0302310B583F311880E4B5B686A
:1023400013F4006314D0F1EE103AEFF309844FF068
:102350008073683CE361094BDB6B236684F3098877
:10236000FFF7FAFB10B1064BA36110BD054BFBE76D
:1023700083F31188F9E700BF00ED00E000EF00E013
:102380002F0400083204000870B5BFF34F8FBFF36D
:102390006F8F1A4A0021C2F85012BFF34F8FBFF35C
:1023A0006F8F536943F400335361BFF34F8FBFF313
:1023B0006F8FC2F88410BFF34F8FD2F8803043F68E
:1023C000E074C3F3C900C3F34E335B0103EA0406B0
:1023D000014646EA81750139C2F86052F9D2203BC4
:1023E00013F1200FF2D1BFF34F8F536943F48033C1
:1023F0005361BFF34F8FBFF36F8F70BD00ED00E0EF
:10240000FEE70000214B2248224A70B5904237D3A4
:10241000214BC11EDA1C121A22F003028B4238BF74
:1024200000220021FEF7F0FC1C4A0023C2F8843091
:10243000BFF34F8FD2F8803043F6E074C3F3C90086
:10244000C3F34E335B0103EA0406014646EA817595
:102450000139C2F86C52F9D2203B13F1200FF2D1AE
:10246000BFF34F8FBFF36F8FBFF34F8FBFF36F8FEC
:102470000023C2F85032BFF34F8FBFF36F8F70BD90
:1024800053F8041B40F8041BC0E700BF902F00085E
:10249000F82F0020F82F0020F82F002000ED00E09A
:1024A00000F01EB9014B586A704700BF000C004095
:1024B000034B002258631A610222DA60704700BFA2
:1024C000000C0040014B0022DA607047000C004015
:1024D000014B5863704700BF000C0040FEE700004E
:1024E00070B51B4B0025044686B058600E468562C9
:1024F0000163FFF7F7FE04F11003A560E562C4E98C
:1025000004334FF0FF33C4E90044C4E90635FFF754
:10251000C9FF2B46024604F134012046C4E90823D2
:1025200080230C4A2565FFF74FFB01230A4AE06030
:1025300000920375684672680192B268CDE9022381
:10254000064BCDE90435FFF767FB06B070BD00BF51
:10255000682F0020202E0008252E0008DD2400080A
:10256000024AD36A1843D062704700BF002D002092
:102570004B6843608B688360CB68C3600B694361C1
:102580004B6903628B6943620B680360704700000C
:1025900008B53C4B40F2FF713B48D3F888200A4312
:1025A000C3F88820D3F8882022F4FF6222F00702C3
:1025B000C3F88820D3F88830344B1A6C0A431A6465
:1025C0009A6E0A439A66324A9B6E1146FFF7D0FF15
:1025D00000F5806002F11C01FFF7CAFF00F5806082
:1025E00002F13801FFF7C4FF00F5806002F15401E9
:1025F000FFF7BEFF00F5806002F17001FFF7B8FF42
:1026000000F5806002F18C01FFF7B2FF00F58060F9
:1026100002F1A801FFF7ACFF00F5806002F1C401F0
:10262000FFF7A6FF00F5806002F1E001FFF7A0FFD1
:1026300000F5806002F1FC01FFF79AFF02F58C7152
:1026400000F58060FFF794FF00F00CF9114BD3F810
:10265000902242F00102C3F89022D3F8942242F073
:102660000102C3F894220522C3F898204FF060526B
:10267000C3F89C20084AC3F8A020BDE80840FFF733
:10268000E3BD00BF00440258000002580045025854
:102690002C2E000800ED00E01F00080308B500F034
:1026A000CDFAFFF779FA0B4BDA6B42F04002DA63AE
:1026B0005A6E22F040025A665B6E074B1A6842F06F
:1026C00008021A601A6842F004021A60BDE8084065
:1026D000FFF7E2BD004502580018024870470000AD
:1026E0000E4B9A6C42F008029A641A6F42F008028C
:1026F0001A670B4A1B6FD36B43F00803D363C722DF
:10270000084B9A624FF0FF32DA6200229A615A63F4
:10271000DA605A6001225A611A6070470045025817
:102720000010005C000C0040094A08B51169D3682C
:102730000B40D9B29B076FEA0101116107D5302325
:1027400083F31188FFF73EFA002383F3118808BD55
:10275000000C0040044BDA6B0243DA635A6E1043FC
:1027600058665B6E704700BF0045025808B53C4B89
:102770004FF0FF31D3F8802062F00042C3F8802090
:10278000D3F8802002F00042C3F88020D3F88020E4
:10279000D3F88420C3F88410D3F884200022C3F82F
:1027A0008420D3F88400D86F40F0FF4040F4FF004D
:1027B00040F4DF4040F07F00D867D86F20F0FF4042
:1027C00020F4FF0020F4DF4020F07F00D867D86FAE
:1027D000D3F888006FEA40506FEA5050C3F8880081
:1027E000D3F88800C0F30A00C3F88800D3F8880043
:1027F000D3F89000C3F89010D3F89000C3F890205D
:10280000D3F89000D3F89400C3F89410D3F8940050
:10281000C3F89420D3F89400D3F89800C3F8981024
:10282000D3F89800C3F89820D3F89800D3F88C0018
:10283000C3F88C10D3F88C00C3F88C20D3F88C002C
:10284000D3F89C00C3F89C10D3F89C10C3F89C20CC
:10285000D3F89C30FEF71AFDBDE8084000F0BEB981
:102860000044025808B50122504BC3F80821504BD0
:102870005A6D42F002025A65DA6F42F00202DA67DC
:102880000422DB6F4B4BDA605A689104FCD54A4A4C
:102890001A6001229A60494ADA6000221A614FF4F4
:1028A00040429A61434B9A699204FCD51A6842F4FB
:1028B00080721A60424B1A6F12F4407F04D04FF4BA
:1028C00080321A6700221A671A6842F001021A6001
:1028D0003B4B1A685007FCD500221A611A6912F0A6
:1028E0003802FBD1012119604FF0804159605A67CD
:1028F000344ADA62344A1A611A6842F480321A6041
:102900002F4B1A689103FCD51A6842F480521A6062
:102910001A689204FCD52D4A2D499A6200225A6306
:10292000196301F57C01DA6301F5E77199635A6473
:10293000284A1A64284ADA621A6842F0A8521A60D1
:102940001F4B1A6802F02852B2F1285FF9D14822D1
:102950009A614FF48862DA6140221A621F4ADA648F
:102960001F4A1A651F4A5A651F4A9A6532231F4A31
:102970001360136803F00F03022BFAD1104A136996
:1029800043F003031361136903F03803182BFAD1E2
:102990004FF00050FFF7DEFE4FF08040FFF7DAFE09
:1029A0004FF00040BDE80840FFF7D4BE0080005162
:1029B000004502580048025800C000F00400000121
:1029C000004402580000FF01008890083220600097
:1029D00063020901470E0508DD0BBF01200000203E
:1029E000000001100910E000000101100020005259
:1029F0004FF0B04208B5D2F8883003F00103C2F8B6
:102A0000883023B1044A13680BB150689847BDE879
:102A10000840FFF78FBC00BF782F00204FF0B04276
:102A200008B5D2F8883003F00203C2F8883023B129
:102A3000044A93680BB1D0689847BDE80840FFF797
:102A400079BC00BF782F00204FF0B04208B5D2F813
:102A5000883003F00403C2F8883023B1044A1369B4
:102A60000BB150699847BDE80840FFF763BC00BF51
:102A7000782F00204FF0B04208B5D2F8883003F02C
:102A80000803C2F8883023B1044A93690BB1D069B6
:102A90009847BDE80840FFF74DBC00BF782F0020E5
:102AA0004FF0B04208B5D2F8883003F01003C2F8F6
:102AB000883023B1044A136A0BB1506A9847BDE8C5
:102AC0000840FFF737BC00BF782F00204FF0B0431D
:102AD00010B5D3F8884004F47872C3F88820A306B0
:102AE00004D5124A936A0BB1D06A9847600604D5A0
:102AF0000E4A136B0BB1506B9847210604D50B4A55
:102B0000936B0BB1D06B9847E20504D5074A136C61
:102B10000BB1506C9847A30504D5044A936C0BB1D4
:102B2000D06C9847BDE81040FFF704BC782F002018
:102B30004FF0B04310B5D3F8884004F47C42C3F89A
:102B40008820620504D5164A136D0BB1506D984765
:102B5000230504D5124A936D0BB1D06D9847E0045C
:102B600004D50F4A136E0BB1506E9847A10404D5DB
:102B70000B4A936E0BB1D06E9847620404D5084A95
:102B8000136F0BB1506F9847230404D5044A936F19
:102B90000BB1D06F9847BDE81040FFF7CBBB00BF2B
:102BA000782F002008B50348FEF7F6FCBDE8084082
:102BB000FFF7C0BB2424002008B50348FEF7ECFC57
:102BC000BDE80840FFF7B6BB9024002008B5FFF72A
:102BD000ABFDBDE80840FFF7ADBB0000062108B51E
:102BE0000846FEF75FFD06210720FEF75BFD062184
:102BF0000820FEF757FD06210920FEF753FD0621A8
:102C00000A20FEF74FFD06211720FEF74BFD062197
:102C10002820FEF747FD09217A20FEF743FD072112
:102C20003220FEF73FFD0C215220FEF73BFD0C2128
:102C30005320BDE80840FEF735BD000008B5FFF79A
:102C400095FD00F009F8FEF7EBFEFFF747FDBDE844
:102C50000840FFF725BC00000023054A1946013350
:102C6000102BC2E9001102F10802F8D1704700BF31
:102C7000782F002010B501390244904201D1002084
:102C800005E0037811F8014FA34201D0181B10BDD5
:102C90000130F2E753544D333248373F3F3F005342
:102CA000544D3332483733782F3732780053544DF0
:102CB0003332483734332F3735332F373530000030
:102CC00001105A000310590001205800032056003B
:102CD00010000240080002400008024000000B0003
:102CE00028000240080002400408024006010C00CF
:102CF00040000240080002400808024010020D0097
:102D000058000240080002400C08024016030E0062
:102D1000700002400C0002401008024000040F0046
:102D2000880002400C000240140802400605100012
:102D3000A00002400C0002401808024010061100DA
:102D4000B80002400C0002401C08024016072F0089
:102D50001004024008040240200802400008380025
:102D600028040240080402402408024006093900F1
:102D7000400402400804024028080240100A3A00B9
:102D800058040240080402402C080240160B3B0085
:102D9000700402400C04024030080240000C3C0069
:102DA000880402400C04024034080240060D44002E
:102DB000A00402400C04024038080240100E4500F6
:102DC000B80402400C0402403C080240160F4600C2
:102DD000009600000000000000000000000000005D
:102DE000000000000000000000000000E1190008E1
:102DF000CD190008091A0008F5190008011A000881
:102E0000ED190008D9190008C5190008151A00089D
:102E100063300000102E0008582D0020682F00207D
:102E20006D61696E0069646C650000000000002837
:102E300000000000AAAAAAAA00000024FFFF0000C8
:102E40000000000000000000000000000000000082
:102E5000AAAAAAAA00000000FFFF000000000000CC
:102E6000000000000000000000000000AAAAAAAABA
:102E700000000000FFFF0000000000000000000054
:102E80000000100000000000AAAAAAAA000000008A
:102E9000FFFF000000000000000000000A800200A8
:102EA00000000000AAAAAAAA05400100FFFF000036
:102EB0008800007007000000000000000000000013
:102EC000AAAAAAAA00000000FFFF0000000000005C
:102ED000000000000000000000000000AAAAAAAA4A
:102EE00000000000FFFF00000000000000000000E4
:102EF0000000000000000000AAAAAAAA000000002A
:102F0000FFFF0000000000000000000000000000C3
:102F100000000000AAAAAAAA00000000FFFF00000B
:102F200000000000000000000000000000000000A1
:102F3000AAAAAAAA00000000FFFF000000000000EB
:102F4000000000000000000000000000AAAAAAAAD9
:102F500000000000FFFF0000000000000000000073
:102F60002E0400000000000000001A000000000015
:102F7000FF0000002424002000000000942C000822
:102F8000830400009F2C000850040000AD2C0008B2
:00000001FF
